S02100002E2E5C62696E5C64656D6F70726F675F73746D3332663330332E7372656345
S3150800200000300020592F0008A72F0008A92F000824
S31508002010AB2F0008AD2F0008AF2F00080000000006
S31508002020000000000000000000000000B12F0008BA
S31508002030B32F000800000000B52F0008753000080F
S31508002040B92F0008BB2F0008BD2F0008BF2F0008B6
S31508002050C12F0008C32F0008C52F0008C72F000886
S31508002060C92F0008CB2F0008CD2F0008CF2F000856
S31508002070D12F0008D32F0008D52F0008D72F000826
S31508002080D92F0008DB2F0008DD2F0008DF2F0008F6
S31508002090E12F0008E32F0008E52F0008E72F0008C6
S315080020A0E92F0008EB2F0008ED2F0008EF2F000896
S315080020B0F12F0008F32F000800000000F52F000894
S315080020C0F72F00080000000000000000F92F0008A4
S315080020D000000000FB2F0008FD2F0008FF2F000856
S315080020E0013000080330000800000000000000006E
S315080020F000000000000000000000000000000000D2
S3150800210000000000000000000000000000000000C1
S315080021100000000000000000053000080730000835
S3150800212000000000000000000000000000000000A1
S315080021300000000000000000000000000000000091
S31508002140093000080B3000080000000000000000FD
S315080021500000000000000000000000000000000071
S315080021600000000000000000000000000000000061
S315080021700000000000000000000000000000000051
S31508002180000000000D300008EE11AA5510B5054CE8
S31508002190237833B9044B13B10448AFF30080012305
S315080021A0237010BD9C00002000000000503100087C
S315080021B0084B10B51BB108490848AFF3008008481A
S315080021C0036803B910BD074B002BFBD0BDE81040D0
S315080021D0184700BF00000000A0000020503100088A
S315080021E09C00002000000000154B002B08BF134B75
S315080021F09D46A3F5803A00218B460F461348144A9C
S31508002200121A00F079FF0F4B002B00D098470E4B9F
S31508002210002B00D098470020002104000D000D482F
S31508002220002802D00C48AFF3008000F03FFF2000E2
S31508002230290000F087FE00F025FF00BF0000080017
S315080022400030002000000000000000009C00002074
S315080022500C0100200000000000000000F0B500247A
S3150800226022E0134D15F814E005EB44056F780EEBE4
S31508002270070606FB00064FF4FA4595FBF6F506FB3E
S3150800228005F5B5F5FA4F0DD195FBF6F6B6B20E8003
S31508002290013EB6B2B6F5806F04D282F800E01F7030
S315080022A00120F0BD0134E4B2112CDAD90020F0BDCA
S315080022B02431000870B588B001214FF4003000F0D1
S315080022C045FD01214FF4003000F032FD07220221BE
S315080022D04FF0904000F066FB07220F214FF0904028
S315080022E000F060FB00248DF81E4001258DF81F5074
S315080022F002268DF81C600423069303238DF81D30EF
S3150800230006A94FF0904000F001FB8DF81C604FF4D1
S315080023100043069306A94FF0904000F0F7FA4FF4F1
S315080023206143009301940294039405940C23049347
S31508002330054C6946204600F025FD2946204600F052
S3150800234085FD08B070BD00BF0044004070B58AB076
S3150800235001214FF4003000F0EBFC09220B214FF06D
S31508002360904000F01FFB09220C214FF0904000F02E
S3150800237019FB4FF4C053089302238DF82430032326
S315080023808DF8253000248DF8264001258DF8275034
S3150800239008A94FF0904000F0B9FA29464FF00070AE
S315080023A000F0D4FC244E304600F028F905A800F0C9
S315080023B03DFA6B460DEB05020DF102014FF4FA707A
S315080023C0FFF74CFF8DF81A408DF81B408DF81C401E
S315080023D08DF81D408DF81E408DF81F408DF816406B
S315080023E08DF817409DF80130013B8DF818309DF89F
S315080023F00030013B8DF81930BDF80230ADF81430C5
S3150800240005A9304600F006F98DF80E408DF80F4004
S315080024108DF81050ADF80440ADF80640ADF8084008
S31508002420ADF80A40ADF80C408DF8115001A800F03F
S3150800243083F90AB070BD00BF0064004010B50446B9
S315080024402021064800F012FD012805D1034800F0B6
S3150800245009FD2070012010BD002010BD0044004079
S3150800246008B5FFF727FFFFF771FF08BDBFF34F8FCA
S315080024700449CA6802F4E062034B1343CB60BFF316
S315080024804F8FFEE700ED00E00400FA0508B5204B83
S315080024901B789BB91F48FFF7D1FF012836D11D4B82
S315080024A01B78002B32D000F0DFFD1B4B1860012291
S315080024B0174B1A700022194B1A7008BD174B1B7858
S315080024C0013314481844FFF7B9FF012814D1134AF9
S315080024D013780133DBB213700E4A1278934215D182
S315080024E000220B4B1A700B4B5B78FF2B0ED1094B56
S315080024F09B785BB9FFF7BAFF00F0B6FD064B1B6881
S315080025006433984202D90022014B1A7008BD00BFF5
S31508002510FA000020B8000020FC000020F900002086
S3150800252000B587B000210D4800F0E2F990B101AA84
S3150800253000210A4800F08AF940F26763019A9A4234
S3150800254008D19DF80F30FF2B04D19DF810300BB938
S31508002550FFF78CFF07B05DF804FB00BF006400407E
S3150800256008B5FFF793FFFFF7DBFF08BD30B583B06B
S3150800257001214FF4802000F0DBFB0825009501239C
S315080025808DF8043000238DF8063003228DF80520D7
S315080025908DF80730054C6946204600F0B7F92946FC
S315080025A0204600F0FDF903B030BD00BF0004004826
S315080025B010B500F059FD0E4B1B68C31AB3F5FA7F28
S315080025C014D304460B4B1B783BB90122094B1A70EE
S315080025D00821094800F0E2F906E00022054B1A70C6
S315080025E00821054800F0DCF9014B1C6010BD00BF4E
S315080025F000010020040100200004004808B501215C
S315080026004FF0007000F0B0FB00214FF0007000F0B2
S31508002610ABFB08BD82B000230193036823F00203D5
S315080026200360036843F00103036002E0019B013382
S315080026300193436813F0010F04D1019A6FF07F43A9
S315080026409A42F3D1436813F0010F6FD08B79012BAF
S3150800265004D1036843F08003036003E0036823F0B2
S3150800266080030360CB79012B04D1036843F0400350
S31508002670036003E0036823F0400303600B7A012B31
S3150800268004D1036843F02003036003E0036823F0E2
S31508002690200303604B7A012B04D1036843F010032F
S315080026A0036003E0036823F0100303608B7A012BB1
S315080026B004D1036843F00803036003E0036823F0CA
S315080026C008030360CB7A012B04D1036843F00403A3
S315080026D0036003E0036823F0040303608A78CB7879
S315080026E01B0643EA82730A7943EA02434A7943EAB4
S315080026F002530A88013A1343C361036823F00103AE
S3150800270003600023019302E0019B013301934368B0
S3150800271013F0010F04D0019A6FF07F439A42F3D168
S31508002720436813F0010F03D0002002E0002000E008
S31508002730012002B0704700BF70B4837A012202FA02
S3150800274003F3394AD2F8001241F00101C2F8001227
S31508002750D2F81C12DC432140C2F81C12027BB2B923
S31508002760314AD2F80C122140C2F80C12817AC68876
S31508002770458845EA0645483142F83150857A8688C3
S31508002780018841EA0641483502EBC5025160027BE1
S31508002790012A16D1244AD2F80C121943C2F80C128F
S315080027A0817A0688458845EA0645483142F8315017
S315080027B0857A8688C18841EA0641483502EBC50212
S315080027C05160C27A32B91849D1F804222240C1F8B8
S315080027D0042205E01449D1F804221A43C1F8042258
S315080027E002892AB91049D1F814221440C1F81442B2
S315080027F00289012A05D10C49D1F814221A43C1F8D5
S315080028001422427B012A05D10749D1F81C22134319
S31508002810C1F81C32044AD2F8003223F00103C2F888
S31508002820003270BC704700BF00640040002383710B
S31508002830C371037243728372C3728370C3700323B6
S3150800284003710223437101230380704710B401F119
S315080028501B031B01C35803F00403DBB2137233B91D
S3150800286001F11B031B01C3585B0D136005E001F161
S315080028701B031B01C358DB08536001F11B031B0133
S31508002880C418C35803F002035372636803F00F03B6
S31508002890937263681B0AD37400EB0113D3F8B8412B
S315080028A0D472D3F8B841240A1473D3F8B841240C67
S315080028B05473D3F8B841240E9473D3F8BC41D47337
S315080028C0D3F8BC41240A1474D3F8BC41240C5474BC
S315080028D0D3F8BC311B0E937421B9C36843F02003A7
S315080028E0C36003E0036943F02003036110BC70472B
S315080028F019B9C06800F003007047012903D10069BF
S3150800290000F0030070470020704700BF70B4002332
S315080029103FE001229A400C68A24339D10A79013A6C
S31508002920D2B2012A1CD885685A000324944025EAA5
S315080029300404846085684C7904FA02F22A438260AA
S315080029408488A5B29AB20124944025EA04048480B6
S315080029508588ADB28C7904FA02F22A4392B2828053
S3150800296004685A00032505FA02F624EA06040460F8
S3150800297006680C79944034430460C4689EB27600B5
S31508002980B54024EA0505CC7904FA02F22A43C26066
S3150800299001330F2BBDD970BC704700BF81617047EA
S315080029A00185704730B401F007039B009A40C908B7
S315080029B0083150F821400F2505FA03F324EA0303EA
S315080029C040F8213050F821301A4340F8212030BC15
S315080029D0704700BFF0B5A04B5B6803F00C03042BEF
S315080029E006D0082B08D003BB9C4B036000241FE0CD
S315080029F09A4B036000241BE0974B5C685A68C4F343
S31508002A008344A31C12F4803F03D1954C04FB03F4C2
S31508002A1009E0914AD26A02F00F0201328F4CB4FBE8
S31508002A20F2F404FB03F4046002E08C4B0360002418
S31508002A30894D6B68C3F30313DFF828E21EF80370A9
S31508002A40FFB2026822FA07F343606968C1F30221FC
S31508002A501EF80110C9B223FA01F181606E68C6F347
S31508002A60C2261EF80660F6B2F340C360ED6A2D0969
S31508002A7005F00F0CDFF8F0E13EF81CE01FFA8EFEB9
S31508002A8015F0100F06D0BEF1000F03D0B4FBFEF50B
S31508002A90056100E00261704DED6A6D0A05F00F0CE4
S31508002AA0DFF8C4E13EF81CE01FFA8EFE15F0100FA1
S31508002AB006D0BEF1000F03D0B4FBFEF5456100E079
S31508002AC04261654D2D6B15F0100F02D1634D85617E
S31508002AD000E08261604D2D6B15F0200F02D15F4D2D
S31508002AE0C56100E0C2615C4D2D6B15F0400F02D147
S31508002AF05A4D056200E00262574D2D6B15F4807F32
S31508002B0006D0944204D1B74202D16500456200E07E
S31508002B104362514D2D6B15F4805F06D0944204D163
S31508002B20B74202D16500856200E083624A4D2D6B8B
S31508002B3015F4007F06D0944204D1B74202D165004D
S31508002B40C56200E0C362444D2D6B15F4806F06D054
S31508002B50944204D1B74202D16500C56400E0C3645B
S31508002B603D4D2D6B15F4006F06D0944204D1B74243
S31508002B7002D16500056500E00365374D2D6B15F438
S31508002B80005F06D0944204D1B74202D1650045657C
S31508002B9000E00365304D2D6B15F4004F06D09442C6
S31508002BA004D1B74202D16400846500E083652A4BEC
S31508002BB01B6B13F0030F01D1816319E0264B1B6BC6
S31508002BC003F00303012B01D1826311E0224B1B6B37
S31508002BD003F00303022B03D14FF40043836307E09A
S31508002BE01D4B1B6B03F00303032B01D11B4B8363A4
S31508002BF0194B1B6B13F4403F01D1C1631CE0164B04
S31508002C001B6B03F44033B3F5803F01D1C26313E075
S31508002C10114B1B6B03F44033B3F5003F03D14FF45C
S31508002C200043C36308E00C4B1B6B03F44033B3F556
S31508002C30403F01D1094BC363074B1B6B13F4402F6D
S31508002C4001D1016426E0044B1B6B03F44023B3F562
S31508002C50802F0BD102641DE00010024000127A009A
S31508002C6000093D0020000020000000202E4B1B6BB1
S31508002C7003F44023B3F5002F03D14FF40043036454
S31508002C8008E0294B1B6B03F44023B3F5402F01D111
S31508002C90264B0364244B1B6B13F4401F01D141647C
S31508002CA01CE0214B1B6B03F44013B3F5801F01D1C5
S31508002CB0426413E01C4B1B6B03F44013B3F5001F6F
S31508002CC003D14FF40043436408E0174B1B6B03F42E
S31508002CD04013B3F5401F01D1144B4364124B1B6BD1
S31508002CE013F4400F01D18164F0BD0F4B1B6B03F445
S31508002CF04003B3F5800F01D18264F0BD0A4B1B6B0C
S31508002D0003F44003B3F5000F03D14FF40043836483
S31508002D10F0BD054B1B6B03F44003B3F5400F01D11F
S31508002D20024B8364F0BD00BF0010024000127A0017
S31508002D3021B1054B5A69104358617047024A5369D5
S31508002D4023EA0000506170470010024021B1054B8C
S31508002D50DA691043D8617047024AD36923EA00004A
S31508002D60D06170470010024021B1054B1A69104323
S31508002D7018617047024A136923EA00001061704718
S31508002D800010024030B599B004460D46036823F09A
S31508002D9001030360436823F440528B68134343607E
S31508002DA0036823F4B05222F00C024968EB68194311
S31508002DB02B690B4313430360836823F440726B69E2
S31508002DC01343836001A8FFF705FE1C4B9C4201D103
S31508002DD00F9A0FE01A4B9C4201D1109A0AE0194B40
S31508002DE09C4201D1119A05E0174B9C4201D1129AD7
S31508002DF000E0139A236813F4004F06D0520029689E
S31508002E00B2FBF1F301FB132204E02968B2FBF1F3EC
S31508002E1001FB13222968B2EB510F00D30133226854
S31508002E2012F4004F06D0C3F3420223F00F031B042B
S31508002E301B0C13439BB2A38119B030BD0038014067
S31508002E400044004000480040004C004021B103689F
S31508002E5043F0010303607047036823F0010303602E
S31508002E60704700BF808CC0F308007047C3690B42E7
S31508002E7001D0012070470020704700BF1222164B70
S31508002E801A60A3F580535A685A605A685A605A6895
S31508002E9042F480625A605A6822F47C125A605A6870
S31508002EA042F460125A601A6842F080721A600B4B3C
S31508002EB01B6813F0007FFAD0084B5A6822F0030209
S31508002EC05A605A6842F002025A60044B5B6803F083
S31508002ED00C03082BF9D1704700200240001002406D
S31508002EE008B5124B1A6842F001021A605968104A6E
S31508002EF00A405A601A6822F0847222F480321A60F4
S31508002F001A6822F480221A605A6822F4FE025A606D
S31508002F10DA6A22F00F02DA62196B064A0A401A6365
S31508002F2000229A60FFF7AAFF08BD00BF0010024002
S31508002F300CC07FF8CCFC00FF08B5FFF717FB00F0C4
S31508002F4071F808BD08B5FFF7F7FFFFF789FAFFF72D
S31508002F502FFBFFF705FBFAE707498D460749084A9D
S31508002F60084B9A42BEBF51F8040B42F8040BF8E727
S31508002F700548804705480047003000205C310008B6
S31508002F80000000209C000020E12E0008E92100082E
S31508002F901F49204A002301E041F8043B9142FBD334
S31508002FA0FFF7D0FFFEE7FEE7FEE7FEE7FEE7FEE7F0
S31508002FB0FEE7FEE7FEE7FEE7FEE7FEE7FEE7FEE7DB
S31508002FC0FEE7FEE7FEE7FEE7FEE7FEE7FEE7FEE7CB
S31508002FD0FEE7FEE7FEE7FEE7FEE7FEE7FEE7FEE7BB
S31508002FE0FEE7FEE7FEE7FEE7FEE7FEE7FEE7FEE7AB
S31508002FF0FEE7FEE7FEE7FEE7FEE7FEE7FEE7FEE79B
S31508003000FEE7FEE7FEE7FEE7FEE7FEE7FEE700006F
S315080030109C0000200C010020014B1860704700BF7F
S315080030200801002008B50C4B1B680C4AA2FB0323B9
S315080030309B09013BB3F1807F09D2094A5360F0210D
S31508003040084B83F82310002393600723136000209E
S31508003050FFF7E2FF08BD00BF30000020D34D621025
S3150800306010E000E000ED00E0014B1868704700BF73
S3150800307008010020024A136801331360704700BF35
S315080030800801002008B5074B044613B10021AFF329
S315080030900080054B1868836A03B19847204600F0FC
S315080030A033F800BF000000004C31000870B50E4B25
S315080030B00E4CE41AA41000251E46A54204D056F864
S315080030C0253098470135F8E700F020F8084C094BF9
S315080030D0E41AA41000251E46A54204D056F8253049
S315080030E098470135F8E770BD940000209400002049
S315080030F0980000209400002002440346934202D020
S3150800310003F8011BFAE77047FEE70000F8B500BFB1
S31508003110F8BC08BC9E467047F8B500BFF8BC08BCAA
S315080031209E467047050206020603070308030903BD
S3150800313009040A040B040C040C050D050E050F05FD
S315080031400F06100610071008430000003400002080
S30908003150000000006D
S30D0800315494F0FF7F0100000062
S3150800315C010002000400060008000A000C0010001A
S3150800316C2000400080000001000000000000000064
S3150800317C0000000001020304010203040607080903
S3150800318C0090D003000000000000000000000000C2
S3150800319C0000000000000000000000000000000015
S315080031AC0000000048310008000000000000000084
S315080031BC00000000000000000000000000000000F5
S315080031CC00000000000000000000000000000000E5
S315080031DC00000000000000000000000000000000D5
S311080031EC00000000B12100088D21000839
S70508002000D2
